:020000040800F2
:1000000070210020B5010008F9010008B51A0008A8
:10001000F9010008F9010008F901000800000000DA
:10002000000000000000000000000000F9010008CE
:10003000F901000800000000F9010008F9010008BA
:10004000F9010008F9010008F9010008F9010008A8
:10005000F9010008F9010008F9010008F901000898
:10006000F9010008F9010008F9010008F901000888
:10007000F9010008F9010008F9010008F901000878
:10008000F9010008F9010008F9010008F901000868
:10009000F9010008F9010008F9010008F901000858
:1000A000F9010008F9010008F9010008F901000848
:1000B000F9010008F9010008F9010008D11500084C
:1000C000DD150008E9150008F5150008F90100081C
:1000D000F9010008F9010008F9010008F901000818
:1000E000F9010008F9010008F9010008F901000808
:1000F000F9010008F9010008F9010008F9010008F8
:10010000F9010008F9010008F9010008F9010008E7
:10011000F9010008F9010008F9010008F9010008D7
:10012000F9010008F9010008F9010008F9010008C7
:10013000F9010008F9010008F9010008F9010008B7
:10014000F9010008F9010008F9010008F9010008A7
:10015000F9010008F9010008F9010008F901000897
:10016000F9010008F9010008F9010008F901000887
:10017000F9010008F9010008F9010008F901000877
:04018000F901000879
:100184008BB8185876342E332D616C706861322D1B
:1001940033342D6738663564383732000000000088
:0F01A40000000000386635643837320000000173
:1001B400002103E00A4B5B584350043109480A4BC1
:1001C40042189A42F6D3094A02E0002342F8043B5B
:1001D400074B9A42F9D301F0EBFF01F09BFC704707
:1001E4004436000800000020140000201400002001
:1001F4006C010020FEE7000030B501208BB002F056
:1002040021FC002401902546E0B200F049FC01AA3B
:1002140008B9105519E0135D042B10DD164800F0E1
:1002240035FE02A92022019801F08DFF02A800F0FA
:100234002DFE0120002102F0F5FB00201AE001331D
:10024400DBB2052B135528BF01250134042CDBD167
:10025400019C54B1094800F019FE204602A920224D
:1002640001F071FF02A800F011FE0120214602F006
:10027400D9FB28460BB030BD482E0008742E000868
:1002840008B500F017FB80F00100C0B208BD000003
:1002940008B54FF48061034802F0B1F9003018BF8B
:1002A400012008BD001802402DE9F0434A4C89B0F2
:1002B400204600F005FE20460D21052202F0AAF991
:1002C40020460E21052208AE02F0A4F9052220469C
:1002D4000C2102F09FF94FF4005346F81C3D002511
:1002E40001274FF00209204631468DF80A508DF857
:1002F4000B508DF808908DF8097002F03FF94FF417
:10030400804320463146019302F038F94FF480537C
:100314002046314601934FF4007802F02FF920462D
:1003240031468DF808508DF80B70CDF8048002F03A
:1003340025F94FF480632046314601938DF8085027
:100344008DF80B5002F01AF94FF4807320463146B1
:1003540001938DF808708DF80B5002F00FF94FF4EB
:1003640000432046314601938DF80A708DF80B50F6
:1003740002F004F939464FF4001002F0F7FAA4F53C
:100384004444164B164E1E60204602F06BFB03A835
:1003940002F0DFFB4FF4827339463046ADF80E307D
:1003A400ADF80C50ADF81050ADF81290ADF81470D3
:1003B400ADF8168001F024F903A9ADF81800204621
:1003C400ADF81A5002F0A6FB2046394602F0CDFBE8
:1003D40009B0BDE8F08300BF0018024014000020FB
:1003E4000024F40008B5022001F097FE012000F07B
:1003F40045FB022001F091FE0120BDE8084000F019
:100404002BBB000010B504460548022102F0BEFBD8
:100414000028F9D021460248BDE8104002F0B4BBE0
:100424000054014038B5012204460D4629484FF4D2
:10043400807102F0EAF8012001F06FFE25484FF4C4
:100444000041002202F0E1F84FF4807100222148BB
:1004540002F0DBF8012001F060FE4FF400411D487A
:10046400012202F0D2F8012001F057FE19484FF49E
:10047400007102F0C4F818B11748184A6A210AE05A
:1004840014484FF4004102F0BAF808B1254404E0DE
:100494001148134A6B2101F0B3FDAC4204D014F8A7
:1004A400010BFFF7AFFFF8E70A484FF48071012210
:1004B40002F0ABF808240020FFF7A4FF013CFAD1B6
:1004C4004FF40071034802F09AF8003018BF01207D
:1004D40038BD00BF001802408D2E0008972E00087A
:1004E400B22E000810B504460B4802F04AFB0A4835
:1004F400022102F04BFB0028F9D00748214602F004
:1005040043FB0548012102F041FB0028F9D00248D1
:1005140002F037FBC0B210BD0054014010B54FF4D7
:10052400807104460022054802F06FF8642001F04F
:10053400EFFD2046BDE81040FFF764BF00180240FD
:1005440008B50748802102F021FB0028F9D10548AD
:100554004FF480710122BDE8084002F056B800BF94
:10056400005401400018024010B540F2F514FFF7A2
:100574008FFE50B1013C04D1054800F087FC2046B1
:1005840010BD642001F0C4FDF1E7012010BD00BFDF
:10059400CF2E000810B5224C638822884FF6FF71D5
:1005A400DB438A429BB20BD09A4209D11D4800F02A
:1005B4006DFC1D482188FFF735FF20B1012010BDD7
:1005C4001A4800F063FC1A4800F060FC19484FF424
:1005D4008071012202F019F84FF4004100221548FD
:1005E40002F013F8012001F098FD12484FF4004185
:1005F400012202F00AF840F2E9340E484FF4007187
:1006040001F0FDFF0028D9D1013C04D10A4800F0D3
:100614003DFC204610BD642001F07AFDEDE700BFEB
:1006240000000F60F22E000804000F601E2F000867
:100634003A2F000800180240502F000810B5044655
:100644000420FFF76BFF2046FFF7DCFEBDE81040F7
:10065400FFF776BF10B504460120FFF75FFFE0B255
:10066400FFF7D0FEC4F30720FFF7CCFEC4F3074026
:10067400FFF7C8FE200EFFF7C5FEBDE81040FFF7E8
:100684005FBF000010B5FFF70FFEFFF783FF08B947
:10069400224830E0224800F0DDFB4FF48071002254
:1006A400204801F0B2FF642001F032FD0020FFF782
:1006B40019FF4FF48071012204461A4801F0A5FF86
:1006C400204600F0F1FB184800F0E0FBFFF78AFE3B
:1006D40000240120FFF7B2FFFFF746FF78B10320A3
:1006E400FFF71CFFFFF72CFF104800F0B3FB204678
:1006F40000F0DAFB0E48BDE8104000F0C7BB01343F
:10070400FFF748FF152CE4D10A4800F0BFFB022094
:10071400FFF704FFBDE81040FFF712BF6C2F00087D
:100724009B2F000800180240C4350008AA2F0008B7
:10073400C52F0008CF2F000808B55D235843094B87
:100744004A1C00EB52001A78B0FBF1F0C0B28242AE
:1007540007D01870FFF77EFF0220BDE80840FFF7BE
:100764006DBF08BD0000002008B5FFF773FF03202C
:10077400BDE80840FFF762BF08B50220FFF7CEFED0
:10078400BDE80840FFF7DCBE01F1C04102F074BAD5
:1007940070B543489AB000F093FB424800F090FBD8
:1007A400414800F08DFB414B93E8030001AD85E81F
:1007B40003003C48294601F0E1FE3A4804210122A5
:1007C40001F023FF00240223029435488DF80830F9
:1007D400072103230C228DF80930019401F01AFF3C
:1007E40080232F480193294601F0C8FE022C04D02F
:1007F4002C48A1B20C2201F00DFF0134102CF5D1CC
:100804004FF6FB7327480193294601F0B7FE0226F1
:100814003146013624480C22B6B201F0FBFE102EFC
:10082400F6D14FF6FC7329461F48019301F0A6FE4A
:10083400042100221B481E4D01F0E7FE0A2001F0AE
:1008440067FC01220421174801F0DFFE1E2001F09D
:100854005FFC0120014602F071F80FCD03AC0FC418
:1008640095E8070084E80700402200210AA802F066
:100874000EFA02230B9308230C934FF48053129324
:100884004FF4005313930AA803AB18930D9601F089
:10089400FBFD0020012101F061FE1AB070BD00BF14
:1008A40000040240000C024000100240A42C000886
:1008B400AC2C00080D4B98221A80A3F68A231B88BF
:1008C400DBB2512B0CD10A4B1B88DBB2522B07D164
:1008D400084B1888C0B2A0F159035842584100E0AF
:1008E4000020024BF0221A80704700BFAA0A006061
:1008F400220000602400006002460B4604205021C0
:1009040000F045BE02460B460420502100F054BEC0
:10091400032873B50E4603D0042804D001F086FBE7
:1009240014241C4D01E01C4D162420460DF1070132
:10093400FFF7E2FF08B900202AE02B78AEB10BB133
:10094400013323E09DF8071021F0060141F0020174
:1009540020468DF80710FFF7D5FF0028EBD00124BF
:1009640003202C7001F0D9FB11E05AB2012A0CDCEF
:100974009DF80710204601F0F9018DF80710FFF7E4
:10098400C1FF0028D7D02E7001E0013B2B7001205D
:1009940002B070BD180000201900002073B525486E
:1009A40000F08EFA02254FF410730024012621482A
:1009B400009369468DF804508DF805508DF8066053
:1009C4008DF8074001F0DAFD1A480621042201F0EF
:1009D40021FE04220921174801F01CFE154800F0ED
:1009E40087FA154800F06CFA42F20C036946124883
:1009F40000938DF805508DF804608DF806408DF84D
:100A0400074001F0BBFD0C4800F072FA042000F02E
:100A140057FD20466946FFF76FFF9DF80050B54229
:100A240005D103202946FFF773FF284600E020463E
:100A340002B070BD000402400014024010B5044628
:100A4400042000F03DFD21460420FFF761FF04204F
:100A5400BDE8104000F066BD38B5074C0546204699
:100A640000F02EFA20462A46042101F0CEFD20464D
:100A7400BDE8384000F03CBA0014024038B5074CD9
:100A84000546204600F01CFA20462A46082101F0BB
:100A9400BCFD2046BDE8384000F02ABA00140240EC
:100AA40038B5094C04EB00146568284600F008FAD0
:100AB4002189284601F0A3FD0446284600F018FACF
:100AC400B4FA84F0400938BDC82C000838B50024B5
:100AD4002546E0B2FFF7E4FFA04001340543042CAF
:100AE400EDB2F6D1284638BDF7B54FF48040012168
:100AF400134C01F03BFF04F140076568284600F001
:100B0400DFF9684601F072FD02238DF80530A37BFE
:100B14008DF807302846A3680093694600268DF8AF
:100B24000460103401F02AFD284600F0E1F9BC42CB
:100B3400E3D14FF48040314601F018FF03B0F0BD1B
:100B4400C82C000808B5054B1B781BB90448322192
:100B540001F062FABDE8084001F0D6BB1A0000209B
:100B640002300008124B1B7870B505460C461BB9C1
:100B74001048382101F050FA032906D98E0831466D
:100B8400FFF7E0FFB6003544A41B6CB12B462C44A0
:100B94000020A34204D013F8012B42EA0020F8E716
:100BA400BDE8704001F0AABBBDE8704001F0BABBDB
:100BB4001A00002002300008024B1A780AB90122F8
:100BC4001A7070471A00002008B5084B1A781AB931
:100BD40007482B2101F020FA01214FF4805059706D
:100BE40001F0A0FEBDE8084001F082BB1A0000201D
:100BF4000230000808B5074B1A781AB90648512183
:100C040001F00AFA002159704FF48050BDE8084001
:100C140001F088BE1A0000200230000870B50C46AE
:100C24000546A608FFF7D0FF28463146FFF78AFF9E
:100C340004F0030105EB8600FFF794FF0446FFF779
:100C4400D9FF204670BD70B5A0B00D460646FFF72B
:100C5400BBFF2C467119802CA1EB0401684608D90E
:100C64008022FFF791FD68462021FFF76BFF803C4F
:100C7400F0E72246FFF788FD21466846FFF772FF3A
:100C84000446FFF7B7FF204620B070BD0A4B1B781F
:100C940010B504467BB10948402101F0E7FF002864
:100CA400F9D00648214601F0DDFF0448402101F057
:100CB400DDFF0028F9D010BD1C00002000480040D2
:100CC4002DE9F043334D83B06C6804F12E0323F017
:100CD400070300AFADEB030D50238DF80030212343
:100CE4008DF8013000238DF8023003238DF8033092
:100CF40004F121035BBAADF80430274B04F1270853
:100D04006E460DF1060203F11C0153F8040B42F880
:100D1400040B8B42F9D11B78137004F1230922468A
:100D240006F123001D4901F0A7FF31464A46002081
:100D340001F0CEF907F1080304F5927443F8040DA9
:100D4400186846F80900FE23B4FBF3F34344073361
:100D540023F00703ADEB030D31464246684601F02C
:100D64008FF904465520FFF791FF6E466C44A64266
:100D740007D016F8010B552808BF0020FFF786FF9F
:100D8400F5E75520FFF782FF00230C376B60BD4663
:100D9400BDE8F0831C000020102D00082400002072
:100DA4002DE9F041274C86B0204600F089F84FF435
:100DB4008020012101F0CEFD20460A21072201F006
:100DC40029FC06AE072220460B2101F023FC4FF438
:100DD400806346F8183D002501274FF0020820469D
:100DE40031468DF806508DF807708DF804808DF823
:100DF400058001F0C3FB4FF40063204631460093A5
:100E04008DF8048001F0BAFBADF80C50ADF80E502B
:100E1400ADF81050ADF814500B4D0C4B029328460E
:100E24000C2302A9ADF8123001F0B6FE284639466B
:100E340001F00CFF204600F05BF8054B1F7006B074
:100E4400BDE8F081000802400048004040420F0025
:100E54001C00002038B50C4B1A781C469AB1451E6C
:100E640015F8012F7AB163680749FF2B0BD80A2ABA
:100E740002D1FFF725FFF3E70D2A1FBF581C5B18AB
:100E840048601A72ECE738BD1C00002008B5054B19
:100E94001B782BB1FFF7DEFFBDE80840FFF710BF5A
:100EA40008BD00BF1C0000201FB50C2201A901F0E1
:100EB4004AF901A8FFF7CEFF05B05DF804FB000076
:100EC40000F13F4000F57E00C0F3872008280AD8CF
:100ED400054A135C591C11542BB9044901230A6BAC
:100EE400834013430B637047240100200038024001
:100EF40000F13F4000F57E00C0F3872008280DD89C
:100F0400074A135C53B1013BDBB2135433B90549AF
:100F140001230A6B834022EA03030B63704700BF7B
:100F2400240100200038024002460068838823F42C
:100F3400E0631B041B0C838003889BB243F400739F
:100F4400038008230020517513751076704737B558
:100F540004460D46FFF7B4FF0023204669468DF88A
:100F640004308DF805308DF80730009501F006FB4C
:100F74002046FFF7BDFF03B030BD000010B50B4C99
:100F8400342300FB0344236B7BB10A2001F0C5F832
:100F94006068A168FFF7DBFF20696169FFF7D7FF8D
:100FA400236B0120BDE81040184710BD302D000808
:100FB400F7B5044616460F461D46FFF781FF02218A
:100FC40001238DF804108DF805108DF806302046A5
:100FD400002369468DF80730009701F0CFFA2046C8
:100FE40031462A4601F016FB2046FFF781FF03B085
:100FF400F0BD0000027D082A10B5044607D102683E
:10100400938823F4C0631B041B0C938084E0434B3C
:10101400006803EB8203996E01F0CCFB00287BD0BF
:10102400237D072B72D8DFE803F0040B1921323B30
:101034005A6E237A226803F0FE03138201232DE003
:101044002268A37A1382637A0BB1022326E0938881
:101054009BB243F48063938006231FE022681388C5
:101064009BB243F480731380032317E0237A22682E
:1010740043F001031382E37A012B01BF138823F4A5
:1010840080631B041B0C08BF1380042306E0226842
:1010940093889BB243F480639380052323753BE0DC
:1010A40023682269198A237BD154237BE27A013392
:1010B400DBB2591C9142237307D12268138823F4AD
:1010C40080631B041B0C138026E0934224D1226806
:1010D400938823F480631B041B0C938013E0237B0D
:1010E40021692268CB5C1382237BE17A0133DBB272
:1010F4009942237310D1938823F480631B041B0C3F
:1011040093800723CAE72046012101E020460021FD
:10111400BDE81040FFF708BF002010BD302D0008C7
:101124007FB51D4D1C2303FB005306461B790BB9E9
:10113400FFF724FF194C342306FB03446068A168BD
:10114400A289A37BFFF734FF228BA37E2069616908
:10115400FFF72EFFE069012101F0FCFB684601F076
:1011640003FB0F4A236A009393424FF48063ADF864
:101174000A304FF01C0384BF626AADF8062003FBFB
:1011840006F46946285901F085FA2859012101F02D
:10119400F9FA04B070BD00BF30010020302D000802
:1011A400A086010073B504460E460025FFF788FEAD
:1011B4000123204669468DF8043000968DF80550C9
:1011C4008DF8075001F0DAF92046B1B22A4601F051
:1011D4001CFA2046FFF78CFE02B070BD10B5094C16
:1011E400342300FB0344236B5BB100209847606801
:1011F400A168FFF7D7FF20696169BDE81040FFF7D8
:10120400D1BF10BD302D00081C23104A434370B5D4
:1012140005460F4CD058D61801F00EFA342305FBBE
:1012240003440021E06901F095FB337923B9284692
:10123400BDE87040FFF7D2BF6068A168FFF787FE82
:1012440020696169BDE87040FFF781BE300100206C
:10125400302D00082DE9F347504C9A4694F8383065
:10126400884691461BB94E4840F2951104E0042883
:1012740004D94B484FF4CB7100F0CEFE494B1844CF
:101284001C2590F88860754363191B790BB90020FD
:1012940081E063591B8B9F0716D41C2070432718C9
:1012A40000259DF828300B9A87F8089087F80AA043
:1012B40087F80980FB723D733D753A61FD822058C1
:1012C400012101F06BFA2AE03046FFF79DFF30461A
:1012D400FFF726FF6159344B0A8B9007DDD5013B9C
:1012E400FAD1D4E71C2303FB06431B7E23B1019BE5
:1012F4005A1E0192002BF5D11C2303FB0643002246
:101304001A76019903F1100239B3117908291AD117
:1013140055791C2303FB06431B7D082B2BD01C2370
:101324007343E018E1580A8892B242F480720A804A
:10133400E25893889BB243F440739380012303766D
:10134400194B0193D3E7D188B1F57A7F05D20131E6
:10135400D180012000F0E1FEDBE719688B8823F4DB
:10136400E0631B041B0C8B800B889BB243F400735B
:101374000B80082313711C237343E1580A4B0A8B17
:10138400920707D5013BFAD13046FFF73DFF3046BF
:10139400FFF7C6FE284602B0BDE8F0873001002002
:1013A40008300008302D000880841E00017D036889
:1013B400082906D19A8822F480721204120C9A80A9
:1013C40038E09A8A120541BF9A8A22F40062120414
:1013D400120C48BF9A829A8AD20541BF9A8A22F493
:1013E40080721204120C48BF9A829A8A52051ED542
:1013F4009A8A22F480621204120C04299A820AD175
:10140400032202759A8822F4E0621204120C9A8074
:10141400002303760EE0012909D19A8822F4E062C0
:1014240012040021120C01759A80017602E0002159
:10143400FFF77ABD002070472DE9F3411D4C1E4E85
:1014440000251E4F56F8283C44F8043C1C2202FB9D
:1014540005720023237013760822227432788DF8E3
:1014640004204FF001080C2201A82372E371E36009
:101474008DF805208DF806308DF8078000F002FF06
:1014840073788DF8043001A800F0FCFE54F8040CC5
:1014940001F0D2F8454504F11C0406F1340601D0EC
:1014A4004546CEE7284687F83850FFF797FE02B046
:1014B400BDE8F08134010020582D000830010020DF
:1014C40073B5144C94F838200346254622B91248C3
:1014D40040F2331100F0A0FD042807D90522009240
:1014E4000D480E4A40F2351100F08AFD0C4A1344AF
:1014F40093F888401C2303FB04521E46127912B948
:101504002046FFF70DFE06FB0454237901332371B3
:1015140002B070BD30010020083000080E30000811
:10152400302D0008104A08B592F838301BB90F481E
:1015340040F2451104E0042804D90C484FF4A37187
:1015440000F06AFD0A4B18441C2390F8880003FB42
:10155400002213793BB1013BDBB213711BB9BDE827
:101564000840FFF751BE08BD3001002008300008D4
:10157400302D000837B50D4614460093069B0193A1
:1015840001212A462346FFF765FE03B030BD07B5A7
:1015940000930123FFF7EEFF03B05DF804FB37B5BA
:1015A4000D4614460093069B019300212A462346C8
:1015B400FFF750FE03B030BD1FB504AC04F8013D85
:1015C40001230094FFF7EBFF04B010BD0148FFF7BF
:1015D40011BD00BF300100200148FFF7E7BE00BF86
:1015E400300100200148FFF705BD00BF4C01002079
:1015F4000148FFF7DBBE00BF4C010020FFF71EBA15
:1016040030B585B004460D46684601F047F90DB97A
:10161400029805E0012D01D1039801E000F006FDD8
:10162400B4EB500F0ED8B0FBF4F000F080FD0028AE
:1016340002DC0748272103E0082804DD04482821A8
:1016440000F0EAFC01200138C00080B205B030BDD2
:101654003A300008B0F1006F10B504460BD20C48C4
:10166400FFF7F8FB2046FFF71FFC0A48FFF7F2FBE1
:101674004FF0FF3010BD084B002053F8042BA2425A
:1016840002D81A68944202D301300B28F5D110BD58
:10169400B230000840300008C02D00082DE9F8439E
:1016A40006462A480C4617469846FFF7D3FB3046B1
:1016B400FFF7FAFB2648FFF7CDFB2046FFF7F4FBC4
:1016C4002448FFF7C7FBD4B33046FFF7C3FF0546F2
:1016D400601E3044FFF7BEFF002D814632DB002838
:1016E40030DB461B01361FB1002031464246B84765
:1016F40000F02AFE2C464C451FDCF32000F03AFE95
:10170400154B002133F8140000F06CFE09280BD0AF
:101714001248FFF79FFB2046FFF7C6FB1048FFF770
:10172400B5FB00F01FFE0DE02FB1C5F10100204410
:1017340031464246B8470134DDE700F013FE01208C
:10174400BDE8F8830020BDE8F88300BF5B300008E3
:101754006F30000872300008F02D00087630000861
:10176400C43500082DE9F0470646234814460D46C3
:101774001F46FFF76FFB3046FFF796FB1F48FFF746
:1017840069FB2046FFF790FB1D48FFF763FB00F061
:10179400DBFDF32000F0EEFD4FEAD41805EB04095D
:1017A4002C464C45C5EB040A20D0701B204414F889
:1017B400011B00F04DFE09280DD01248FFF74AFB2B
:1017C4003046FFF771FB1048FFF760FB00F0CAFDDD
:1017D4000020BDE8F087002FE3D01AF07F0FE0D19E
:1017E4004FEADA104146089AB847DAE700F0BAFD42
:1017F4000120BDE8F08700BF8E3000086F3000087C
:1018040072300008A2300008C435000808B545F25B
:10181400555000F0DDFF042000F0E0FF40F6FF70BB
:1018240000F0E2FF002000F0D3FF4FF480500121CC
:10183400BDE8084000F07CBD08B500F0E3FFBDE85A
:10184400084000F0D7BF08B57D2001F0D7F800307C
:1018540018BF012008BD4900FEF76EBF4B0803EB1B
:101864005000FEF769BF000070B586B00546FFF76B
:10187400A3F901210020FEF75FFF042000F020FB04
:1018840003A8294600F06EFB03A800F07AFB08B910
:1018940028480BE02848FFF7F9FA05F10C000499F1
:1018A400FFF7D1F9059B984204D02448FFF7EEFADC
:1018B40001203DE0049C2248FFF7E8FA2146214A32
:1018C40021480023FFF7EAFE049E2048FFF7DEFAD2
:1018D400002405F1C0411E4B009432460C311A48D5
:1018E400FFF740FF1B48FFF7B5FA0498FFF7DCFA4F
:1018F4001948FFF7AFFA04991348FFF78FF9054623
:101904001648FFF7A7FA0598FFF7CEFA1448FFF731
:10191400A1FA2846FFF7C8FA1248FFF7B7FA059B61
:101924009D4204D01048FFF7B1FA022000E020469F
:1019340006B070BDBB300008D9300008F63000088E
:10194400193100085B180008004000082C31000819
:10195400611800083F3100084D3100085631000875
:1019640069310008C43500086F31000808B5022049
:1019740000F0BEFAD8B3042000F0BAFA70B11C48E3
:10198400FFF784FA042000F0A7FA022000F0A4FA7A
:101994004FF40040BDE8084000F09EBA1548FFF738
:1019A40075FA082000F098FA102000F095FA20202B
:1019B40000F092FA402000F08FFA4FF48010FFF705
:1019C40053FF022807D1082000F07AFA102000F013
:1019D40077FA00F04DFB042000F07EFA022000F0BC
:1019E4007BFA4FF40040BDE8084000F069BA08BD36
:1019F400BA310008F031000810B52548FFF746FA5F
:101A04004FF40010FFF730FF10B102283AD809E074
:101A1400202000F061FA402000F05EFA802000F0FF
:101A24004FFA2FE0082000F04BFA102000F048FA9B
:101A3400202000F05DFA20B91648FFF727FA20208D
:101A440007E0402000F054FA58B91348FFF71EFA93
:101A5400402000F035FA4FF4007000F031FA00F045
:101A640007FB0E48FFF712FA082000F035FA1020A1
:101A740000F032FA202000F02FFA402000F02CFA77
:101A8400002400E00124042000F026FA204610BDC2
:101A94000B320008253200085E3200089732000835
:101AA40008B50248FFF7F2F900F0E7FAD13200086E
:101AB4001EF0040F0CBFEFF30880EFF30980FFF76B
:101AC400EFBF70471FB504461048FFF7DFF901A9BF
:101AD4000C22204600F037FB01A8FFF7D7F9204677
:101AE400FEF742FEFEF7F2FF094B20F004001870E7
:101AF4001C46FEF7EBFF237800F0FB00834201D085
:101B040000F0B6FA0A2000F008FBF2E7C73200083A
:101B1400690100207FB54FF08050012100F01AFFC9
:101B2400022000F07DFE012807D1022000F082FE91
:101B3400BC48FFF7ABF900F0A0FA00214FF0805049
:101B440000F008FFFFF72CF9B748FFF79FF9B748F3
:101B5400FFF79CF9B648FFF799F9B648FFF796F9ED
:101B6400B548FFF793F9B548FFF790F9B448FFF784
:101B74008DF9B448FFF78AF9B348FFF787F9B348FA
:101B8400FFF784F9FFF758FCFEF708FF00F0BAF9F5
:101B940000F0D0F900210C2201A801F078F800F03F
:101BA400C5F901A90C2200F0CEFA01A8FFF76EF9DD
:101BB4009D48FFF76BF99C48FFF768F94FF48040A4
:101BC40000F096F990B1A248FFF760F94FF4804015
:101BD40000F082F9082000F07FF9102000F07CF971
:101BE400202000F079F9402000F076F9FEF7D0FDCE
:101BF400FEF77AFFFEF746FDFEF7FEFA08B19548B8
:101C040003E0FEF73DFB10B19348FFF75BFF00F0E4
:101C14008CF9802000F06CF918B1802000F05CF998
:101C240056E04FF4003000F063F9044620B14FF45D
:101C3400003000F051F94DE00120FEF731FFB0B162
:101C44002046FEF72DFF90B18448FFF71FF941F2BB
:101C540088340120FEF724FF98B10020FEF720FF0E
:101C640078B1012000F059FA013CF2D132E07C4B0A
:101C74000CCB013301D0013203D17A48FFF706F9C6
:101C840028E0FFF7E0FD48B3FFF7DDFD10B176482B
:101C9400FFF7FCF84FF4007000F02AF910B1734814
:101CA400FFF7F4F84FF4007000F016F9102000F07C
:101CB4001FF9002800F0F0806D48FFF7E7F80820CE
:101CC40000F00AF9102000F007F9FFF795FE98B923
:101CD40068489AE76848FFF7D9F8F6E74FF40070C8
:101CE40000F006F90028CFD1082000F0F5F8102004
:101CF40000F0F2F8FFF73AFE4FF4005000F0F8F865
:101D040004464FF4805000F0F3F8400040EA8400A9
:101D1400C4B24FF4006000F0EBF82043C0B20728CF
:101D2400C3B20DD14FF4006000F0D6F84FF48050E8
:101D340000F0D2F84FF4005000F0CEF84F4864E7BA
:101D44000133DBB2023B4FF40060052B11D8DFE80E
:101D540003F00C1003100C1000F0BEF84FF4805088
:101D640000F0BAF84FF4005003E000F0B5F84FF477
:101D7400805000F0A5F8FFF749FDFFF75DFD384BF3
:101D84003F485D681E68FFF765F82846FFF78CF842
:101D94003C48FFF75FF80022930003F1604303F52A
:101DA400614301324FF0FF31082AC3F88010C3F8B1
:101DB4008011F1D1344B4FF4801200241A635C6318
:101DC4009C631C645C6400F045FD3048012100F014
:101DD400D9FD21462D4800F0D5FDF120012100F068
:101DE400DDFD2146F12000F0D9FD0120014600F07F
:101DF400E1FD2146012000F0DDFD2548012100F030
:101E0400E5FD2146224800F0E1FD2248012100F0D1
:101E1400E9FD2048214600F0E5FD63B64FF0FF3EA2
:101E2400B5462847DC320008C4350008E93200080A
:101E340000330008193300084733000876330008DC
:101E4400A6330008D7330008093400083B340008DF
:101E54006C340008014550FE024550FE99340008D8
:101E640000400008CB340008DE340008F6340008D3
:101E740016350008034550FE8A350008044550FE17
:101E8400A9350008BD350008003802400010E022E2
:101E9400FFC9FEF6337F7704082000F029F820B14B
:101EA4000548FEF7F3FF102003E00448FEF7EEFFB9
:101EB400082000F005F81DE73E35000864350008E9
:101EC40010B50446002000F0BDFD40EA04010020E6
:101ED400BDE8104000F0A6BD10B50446002000F097
:101EE400B1FD20EA04010020BDE8104000F09ABDD5
:101EF40010B50446002000F0A5FD204214BF0120C7
:101F0400002010BD08B54FF08050012100F022FDE3
:101F1400012000F07FFC0120FFF7EAFF20B9012136
:101F2400BDE8084000F07EBD08BD7047022000F007
:101F340089BD000008B5FFF7F9FF054B1968884211
:101F440004D00220BDE8084000F06CBD08BD00BF0D
:101F54008401000808B50248FEF798FF00F088F8ED
:101F6400C53500081FB504460C2201A8FEF70CFC79
:101F740001AB03CB20601868A0602046616004B008
:101F840010BD0068A0F10C0358425841704700008E
:101F940080B50646174610480D461C46FEF75AFF04
:101FA4003846FEF757FF0D48FEF754FF3046FEF75C
:101FB40051FF0B48FEF74EFF2846FEF775FF2CB184
:101FC4000848FEF747FF2046FEF744FF0648FEF7A1
:101FD4005DFFFFF7BFFF00BFE2350008EB350008E7
:101FE400EE350008EC350008C43500081FB506AA14
:101FF40052F8044B039200921A462346FFF7C8FF97
:102004000CB41FB506AA52F8043B03920092014A8D
:10201400FFF7BEFFF035000807B5002300937246B2
:10202400014BFFF7E3FF00BFF7350008744608B51E
:102034000548FEF70FFF2046FEF736FF0348FEF77C
:1020440025FFFFF787FF00BFFF350008C4350008F0
:10205400BFF34F8F0449054BCA6802F4E06213438F
:10206400CB60BFF34F8FFEE700ED00E00400FA05FC
:1020740008B5FEF781FBFFF7EBFF08B5FFF7E8FFB4
:10208400F0B50646002401202546034694421DD09F
:1020940011F804C000F1010EBCF1000F03D1735517
:1020A400774605460DE00133DBB2FF2B774606F891
:1020B40000C007D102F1FF3C644506D07355871C6C
:1020C4007546012301343846E0E770467355F0BD88
:1020D40030B5C9B1C0430A44914213D011F8013B51
:1020E4000A4D83EA000404F00F0455F8244084EAFE
:1020F400101080EA131303F00F0355F8233083EA1A
:102104001010E9E7C04330BD084630BD082E000872
:10211400162358430138FDD1704710B504462CB13D
:102124004FF47A70FFF7F4FF013CF8E710BD10B5E7
:10213400B0FA80F400F027F801280CBFC4F11F00A6
:10214400C4F1200010BD0A2A10B51BDD0C46302353
:1021540004F8023B78234B701C220F239340034066
:10216400D340092B01D8303302E00F2B02D8573368
:10217400DBB200E02023043A04F8013B131DECD148
:1021840000238B7210BD00F0AA33A0EB530000F0C3
:10219400CC3300F0333000EB930000EB101000F070
:1021A4000F3000EB102000EB104000F03F007047B0
:1021B4002D4AD2F8883043F47003C2F888302B4B90
:1021C4001A68002142F001021A6099601A6822F02C
:1021D400847222F480321A60254A5A601A6822F402
:1021E40080221A60D9601A6C224942F080521A6423
:1021F4000A6842F440420A609A689A609A689A604F
:102204009A6842F480529A601B4A5A601A6842F0F3
:1022140080721A601968154A8901FBD5174B40F280
:1022240003611960936823F003039360936843F098
:10223400020393600D4B9A6802F00C02082AF9D14C
:102244009A6822F400029A600D4AC3F884201A683E
:1022540042F080621A60054B1B681B01FBD5024BE0
:102264004FF000629A60704700ED00E000380240D1
:1022740010300024007000401040010F003C024068
:1022840000300050C278037810B512B3164AD168F2
:102294004278C943C1F30221C1F10404E4B2A2406B
:1022A400D4B20F220A4181780A40224303F16043E9
:1022B40003F561431201D2B283F8002303780122AB
:1022C400590903F01F0302FA03F3084A42F82130C4
:1022D40010BD5A09012103F01F03994002F12003A4
:1022E400024A42F8231010BD00ED00E000E100E0D6
:1022F400014B01229A60704700300240014B186084
:10230400186870470030024000EB81018842044B9A
:1023140003D050F8042B1A60F8E71868704700BF20
:1023240000300240014B1868704700BF0030024083
:10233400044B9A6809B1104301E022EA0000986056
:10234400704700BF002004E0044B1A69002ABFBF95
:10235400034A5A6002F188325A607047003C0240D6
:1023640023016745024A136943F000431361704730
:10237400003C0240014BD860704700BF003C024063
:102384000E4BDA68D20310D4DA68D1060FD4DA68B7
:10239400D2050ED4DA6812F0EF0F0CD1DB6813F01B
:1023A400020F14BF0820092070470120704706203F
:1023B4007047022070470720704700BF003C02406E
:1023C40007B509238DF80730FFF7DAFF8DF807000A
:1023D4009DF80730012BF7D09DF8070003B05DF896
:1023E40004FB000070B5064641B1012908D002295A
:1023F4000CBF4FF400754FF4407503E00D4601E047
:102404004FF48075FFF7DCFF09281ED10F4C2369B8
:1024140023F440732361216929432161236923F053
:10242400F8032361236943F002031E4326612369F1
:1024340043F480332361FFF7C3FF236923F00203CE
:102444002361236923F0F803236170BD003C02403B
:1024540070B505460E46FFF7B3FF092811D1094CA4
:10246400236923F44073236123692361236943F0BF
:10247400010323612E70FFF7A3FF236923F00103F7
:10248400236170BD003C024070B543688668856A6C
:102494000468416B46EA0302C3681A4303691A439A
:1024A40043691A4383691A43C3691A43036A1A4383
:1024B400436A1343C26A2B431A43036B1343A200B8
:1024C40002F120420B43082E136002BF136843F04D
:1024D40040031360B1F5801F816B12D18CB14FF0B2
:1024E40020435C681E6846F480161E601E6846F42D
:1024F40080761E600E6924F47004013E44EA06549A
:102504005C608C690B6823434C6843EA04138C6851
:1025140043EA0423CC6843EA04430C69496943EA67
:10252400045343EA0163B5F5804F536010D1C16B86
:1025340088690B680343486843EA0013886843EAE0
:1025440000230869496943EA005343EA016301E04F
:102554006FF07043C2F8043170BD0000800000F1D8
:10256400204019B1036843F0010302E00268024B02
:1025740013400360704700BFFEFF0F00F0B50E6804
:1025840000220123934003EA060E9E452AD15500FA
:1025940003230468AB40DB431C4004600C790768E8
:1025A40004FA05FC013C4CEA0707012C076011D82A
:1025B40084684F791C4084608468AF4027438760F7
:1025C400446824EA0E0444608C7947689440A4B2B9
:1025D4003C434460C4682340C360CB79C468AB40C7
:1025E4002343C3600132102ACBD1F0BD4FF6FF73F1
:1025F40003600023037143718371C37170470369DE
:10260400194214BF0120002070470AB101837047AA
:102614004183704701F00703C90800EB810010B53E
:102624009B00046A0F21994024EA01010162016AB6
:102634009A401143016210BD08B5134B984207D16B
:102644004FF40010012100F0C1F94FF4001014E020
:102654000E4B984207D14FF48000012100F0B6F9E7
:102664004FF4800009E00A4B98420BD14FF400006C
:10267400012100F0ABF94FF400000021BDE808404F
:1026840000F0A4B908BD00BF005400400058004049
:10269400005C00407FB5868826F03F060446360479
:1026A40068460D46360C00F0F9F8029A2C48B2FB45
:1026B400F0F081B20E43A68023882A4E23F0010352
:1026C4001B041B0C23802B68B3420AD85B00013126
:1026D400B2FBF3F39BB2032B89B298BF042321848A
:1026E40023E0EE884BF6FF718E421BBF19214B434A
:1026F40003EB4303B2FBF3F315BF9BB2B2FBF3F35B
:1027040043F480439BB2C3F30B020AB943F00103C1
:102714004FF4967101FB00F24FF47A7192FBF1F2DF
:10272400013292B243F400432284A383238869894B
:10273400AA889BB243F001032380238823F4816396
:1027440023F002031B040A431B0C13439BB2238094
:102754002A89AB8913439BB2238104B070BD00BFA7
:1027640040420F00A086010041F288330360002339
:1027740083804BF6FF72038143814FF48043C28010
:1027840083817047038819B19BB243F0010303E0CE
:1027940023F001031B041B0C03807047038819B149
:1027A4009BB243F4806303E023F480631B041B0C9B
:1027B40003807047838A9AB2038B10B542EA0343BD
:1027C40021F07F4404EA0300431A5842584110BDE3
:1027D400014B1860704700BF00300040014B586047
:1027E400704700BF00300040014B9860704700BF45
:1027F40000300040024B4AF6AA221A60704700BF1C
:1028040000300040024B4CF6CC421A60704700BFC7
:1028140000300040014B1860704700BF20000E429A
:10282400034B5B68184214BF01200020704700BFAF
:1028340000700040064BB0F5402F15BF1A685A6867
:1028440042EA800042F4402214BF18605A60704784
:10285400007000400E4B1A68002142F001021A6019
:1028640099601A6822F0A85222F410221A60094AC8
:102874005A60094AC3F8842002F18062C3F88820B0
:102884001A6822F480221A60D960C3F88C10704749
:102894000038024010300024003000201D4A9368A4
:1028A40003F00C03042B10B503D0082B03D01A4BF0
:1028B40018E01A4B16E05168536811F4800F03F0C6
:1028C4003F03516814BF154A134AB2FBF3F3114A8C
:1028D4005268C2F30142C1F3881101324B435200E2
:1028E400B3FBF2F30B4A036093680D49C3F303137C
:1028F400CC5C0368E34043609468C4F382240C5DB9
:1029040023FA04F484609268C2F342328A5CD340AE
:10291400C36010BD003802400024F40040787D01FB
:1029240001000020044B1A6B09B1104301E022EAB4
:1029340000001863704700BF00380240044B9A6BD4
:1029440009B1104301E022EA00009863704700BF18
:1029540000380240044B1A6C09B1104301E022EA2A
:1029640000001864704700BF00380240044B5A6CE2
:1029740009B1104301E022EA00005864704700BF27
:1029840000380240044B1A6909B1104301E022EAFD
:1029940000001861704700BF00380240044B5A69B8
:1029A40009B1104301E022EA00005861704700BFFA
:1029B40000380240044B9A6909B1104301E022EA4D
:1029C40000009861704700BF00380240044B1A6A47
:1029D40009B1104301E022EA00001862704700BF09
:1029E40000380240044B5A6A09B1104301E022EA5C
:1029F40000005862704700BF003802404209012AB3
:102A0400074B01D11B6803E0022A0CBF1B6F5B6FED
:102A140000F01F0023FA00F000F00100704700BF2F
:102A24000038024082B000230193054B0193019BBF
:102A340003EB80000190019B196002B0704700BF56
:102A44005028004082B000230193054B0193019B61
:102A540003EB80000190019B186802B0704700BF2F
:102A64005028004008B5254B984207D14FF48050B8
:102A74000121FFF7B7FF4FF4805039E0204B984213
:102A840007D14FF480400121FFF7A0FF4FF48040AD
:102A940009E01C4B98420BD14FF400400121FFF791
:102AA40095FF4FF400400021BDE80840FFF78EBFBA
:102AB400154B984207D14FF400500121FFF792FFC4
:102AC4004FF4005014E0114B984207D14FF480109A
:102AD4000121FFF787FF4FF4801009E00C4B984267
:102AE4000BD14FF400100121FFF77CFF4FF40010CD
:102AF4000021BDE80840FFF775BF08BD0030014064
:102B040000380040003C00400034014000500140C7
:102B14000054014003884A8810B503F441540B88DB
:102B240013438A881343CA8813430A8913434A897F
:102B340013438A891343CA89134323439BB20380F3
:102B4400838B23F400631B041B0C83830B8A038293
:102B540010BD0023038043808380C38003814381AD
:102B64008381C381072303827047038819B19BB211
:102B740043F0400303E023F040031B041B0C0380D9
:102B84007047808980B270478181704703891942F8
:102B940014BF0120002070477FB5038ACA889BB206
:102BA40023F440531343038283890E469BB223F4D8
:102BB400B053098923F00C02B3880B4371890B438A
:102BC4009BB213438381838AB2899BB223F44073FB
:102BD4001343838204466846FFF760FE1A4B9C4207
:102BE40003D003F580639C4201D1039D00E0029D64
:102BF400A38931681BB2002B4FF0190202FB05F2C6
:102C0400B4BF4D008D00B2FBF5F5A2896426B5FB77
:102C1400F6F00001010912B2002A06FB1153ADBF00
:102C24001A01D90032313232B5BFB1FBF6F2B2FB30
:102C3400F6F302F0070203F00F03B4BF1043184386
:102C440080B2208104B070BD00100140838919B1A5
:102C54009BB243F4005303E023F400531B041B0C06
:102C640083817047C1F3080181807047038819424A
:102C740014BF01200020704710B5431E0A4491423E
:102C840004D011F8014B03F8014FF8E710BD0244DA
:102C94000346934202D003F8011BFAE77047000091
:102CA4000400000001030000010000000100000016
:102CB40003000000010000000F0000000F000000EE
:102CC40000000000EE2F0008001802401000000071
:102CD40006040000F32F000800180240080000005A
:102CE40006030100F62F000800180240020000004D
:102CF40006010100FD2F0008001802400400000036
:102D040006020100000000000000000001424F4FD5
:102D1400544C4F414445520000000000002A2A0050
:102D2400000000000000000000000000005400400B
:102D340000040240400000000600040000040240B9
:102D4400000200000900040000002000801A0600B0
:102D5400004000001F2000000000000000000000F0
:102D6400005800400014024002000000010004006A
:102D740000140240010000000000040000004000B4
:102D8400801A0600FFBF000021220000000000009E
:102D940001160008010003008200070084000700F8
:102DA400010003000200030040000300800007004C
:102DB400840007000000010000000000000000087B
:102DC400004000080080000800C00008000001085E
:102DD40000000208000004080000060800000808BB
:102DE40000000A0800000C0800000E08000008009B
:102DF400100018002000280030003800400048006F
:102E040050005800000000006410B71DC8206E3B3D
:102E1400AC30D9269041DC76F4516B6B5861B24DDD
:102E24003C7105502083B8ED44930FF0E8A3D6D647
:102E34008CB361CBB0C2649BD4D2D38678E20AA0AF
:102E44001CF2BDBD537475636B20627574746F6E30
:102E540020726567697374657220697320696E7680
:102E6400616C69642C20636C656172696E672E0005
:102E7400427574746F6E206973207075736865642D
:102E840020617420626F6F740069636534306C7004
:102E94002E630043444F4E45206E6F74206C6F7751
:102EA40020647572696E672072657365740043529D
:102EB40045534554206E6F742068696768206475B3
:102EC40072696E6720726573657400446973706C0F
:102ED400617920627573792D776169742074696DE5
:102EE400656F757420657870697265642100436F3D
:102EF4006E6669677572696E672046504741206641
:102F0400726F6D2062697473747265616D20696E8D
:102F140020666C6173682E2E2E004E6F204650473B
:102F2400412062697473747265616D20696E2066F4
:102F34006C6173682E0046616C6C696E6720626117
:102F4400636B20746F204E56434D2E00465047410C
:102F54002043444F4E452074696D656F7574206538
:102F640078706972656421004650474120636F6E32
:102F740066696775726174696F6E206661696C65F4
:102F8400642E204973207468697320612062696724
:102F9400626F6172643F00465047412076657273E8
:102FA400696F6E3A2000446973706C617920696EB0
:102FB400697469616C697A656420616674657220FC
:102FC4000020726574726965732E00446973706CB5
:102FD400617920696E697469616C697A6174696F79
:102FE4006E206661696C65642E004261636B0055F6
:102FF400700053656C65637400446F776E00637290
:10300400632E63006932632E630049324320646592
:1030140076696365204944206F7574206F66206269
:103024006F756E647320256420286D61783A2025BD
:103034006429006F6E007370692E63002069732029
:103044006F7574736964652073797374656D206634
:103054006C6173680D0A0073797374656D5F666CD7
:103064006173685F657261736528002C2000290D07
:103074000A006661696C656420746F20657261730F
:103084006520736563746F72200073797374656D62
:103094005F666C6173685F77726974652800666146
:1030A400696C656420746F2077726974652061644B
:1030B40064726573732000496E76616C696420667E
:1030C40069726D7761726520646573637269707487
:1030D400696F6E2100436865636B73756D6D696E0E
:1030E40067206669726D77617265207570646174BA
:1030F4006500496E76616C6964206669726D7761FA
:1031040072652043524320696E2053504920666CF7
:10311400617368210065726173655F6F6C645F66DB
:1031240069726D776172650077726974655F6E6547
:10313400775F6669726D7761726500436865636B7A
:1031440073756D6D696E6720002062797465730D07
:103154000A00436865636B73756D202D2077616E7B
:10316400746564200020676F7420004F75722069B5
:103174006E7465726E616C20666C61736820636F37
:103184006E74656E747320617265206261642028B8
:10319400636865636B73756D206661696C6564292A
:1031A400212054686973206973207265616C6C799D
:1031B4002062616421004F75722070726576696FB8
:1031C4007573206669726D776172652075706461CC
:1031D4007465206661696C65642C2061626F727429
:1031E400696E67207570646174652E004E65772082
:1031F4006669726D776172652069732061766169B1
:103204006C61626C6521004C6F6164696E67207249
:1032140065636F76657279206669726D7761726530
:10322400004661696C656420746F206C6F61642072
:103234007265636F76657279206669726D77617203
:10324400652C20737472696B65206F6E652E205433
:10325400727920616761696E2E004661696C6564EC
:1032640020746F206C6F6164207265636F76657281
:1032740079206669726D776172652C207374726946
:103284006B652074776F2E205472792061676169B1
:103294006E2E004661696C656420746F206C6F61EA
:1032A40064207265636F76657279206669726D77E2
:1032B4006172652C20737472696B65207468726521
:1032C400652E2053414420574154434800484152FD
:1032D40044204641554C54006578697420737461E8
:1032E4006E64627900205F5F5F5F202020202020D1
:1032F4002020202020202020205F5F002F5C202021
:103304005F605C20202020202020202020202F27E8
:103314005F5F605C005C205C2C5C4C5C5F5C20202C
:1033240020205F5F5F202F5C205C2F5C205C2020CE
:103334005F5F20205F5F20205F5F20205F5F202091
:103344005F5F00205C2F5F5C5F5F205C20202F2785
:10335400205F20605C205C205C205C205C2F5C2073
:103364005C2F5C205C2F5C205C2F5C205C2F5C203D
:103374005C002020202F5C205C4C5C205C2F5C20B7
:103384005C2F5C205C205C205C5F5C205C205C200B
:103394005C5F2F205C5F2F205C205C205C5F5C20E6
:1033A4005C002020205C20605C5F5F5F5F5C205CD1
:1033B4005F5C205C5F5C205C5F5F5F5F2F5C205C18
:1033C4005F5F5F785F5F5F2F275C2F605F5F5F5F8A
:1033D400205C00202020205C2F5F5F5F5F5F2F5CFC
:1033E4002F5F2F5C2F5F2F5C2F5F5F5F2F20205C90
:1033F4002F5F5F2F2F5F5F2F202020602F5F5F5F85
:103404002F3E205C0020202020202020202020206F
:1034140020202020202020202020202020202020A8
:103424002020202020202020202020202020202098
:103434002F5C5F5F5F2F0020202020202020202091
:103444002020202020202020202020202020202078
:103454002020202020202020202020202020202068
:1034640020205C2F5F5F2F004C61737420666972AB
:103474006D7761726520626F6F742077617320735A
:103484007461626C653B20636C6561722073747255
:10349400696B657300486F6C6420646F776E2055A8
:1034A40050202B204241434B20666F7220352073FD
:1034B4006563732E20746F20666F7263652D626F6F
:1034C4006F7420505246004669726D7761726520B0
:1034D400697320657261736564005761746368641D
:1034E4006F6720636175736564206120726573651D
:1034F4007400536F667477617265206661696C75D8
:1035040072652063617573656420612072657365FB
:1035140074004661696C656420746F207374617211
:1035240074206669726D776172652C207374726998
:103534006B652074687265652E004661696C65640C
:1035440020746F207374617274206669726D776180
:1035540072652C20737472696B652074776F2E000A
:103564004661696C656420746F20737461727420A1
:103574006669726D776172652C20737472696B650C
:10358400206F6E652E00466F7263652D626F6F74D7
:10359400696E67207265636F76657279206D6F64FA
:1035A400652E2E2E00426F6F74696E6720666972F5
:1035B4006D77617265204020002E2E2E0D0A0D0AB3
:1035C40000536F667477617265206661696C757209
:1035D400653B20726573657474696E67210041539D
:1035E400534552543A20002020003A004153534599
:1035F4005254004153534552544E002A2A2A20570C
:103604005446200053544D33320053544D3332202A
:103614007065726970686572616C206C6962726150
:103624007279207472697070656420616E206173B0
:10363400736572740043524F414B204F4F4D00004D
:10364400FF0000000001020304010203040607084E
:043654000900000069
:04000005080001B43A
:00000001FF
